:020000040000FA
:1000000000008A014428FF3F6400200091180F205F
:100010000B191C20170827060319970109009110D6
:100020007115F40803197114F30AE7307307031C00
:100030000800F301F40308000B11711F40280000B1
:100040000230F106F118292878089500F601982168
:1000500008007809950075080C1A7705F6009821B4
:100060000310F70C0318771621001C089D142000BC
:1000700078020319080001300318FF30F807080060
:100080007508F600982108002100683099002200C8
:100090009101930122008C0121009501230002307F
:1000A0008C008E01210000308E00FF308C00240077
:1000B00050308C0021009114210050309E000730F8
:1000C0009D0020007C309C00F9309B0020002030F7
:1000D00084008001840A841F6928A5217716711283
:1000E000711771130C18711796019701181498164F
:1000F00018160B178B168B170A30F4007110711C31
:10010000FE331F30F5001E30F4007110711CFE33F9
:100110000C191A320030FB00FB0A7B08063A01304A
:100120000319FB00B621F5000930F400F30171104A
:100130007118F2330C1DFC332300073091002000AE
:10014000BE21A700C62102320A30F5002708F400BC
:10015000F30171107118AE280C19AA280C1DAE28D5
:10016000F501A90803197116711DB4287111D22067
:10017000AB080319B428F11EB4280C1DFA0A0C1997
:10018000FA017A08FC3E031CB4280B30F200FA0195
:10019000F112E03075052A04F50022000030F0006D
:1001A0002000B42872080B00E128EA280029092958
:1001B00019292929392949295929642973297B2988
:1001C0008E290C190800F20AF1133108F400F3012A
:1001D00071100800F11B0A32B10803190732711CB3
:1001E0000532F1177508E0393004F5000C1D0800E0
:1001F000F11F03320930F2000800F116F20A08007C
:100200002108F400F3017110F20AA9080319711210
:100210000800711C080071102208F400F301750831
:10022000E0392C04F500F20A22000430F00020002E
:100230000800711C080071102308F400F301750810
:10024000E0392D04F500F20A22000830F000200009
:100250000800711C080071102408F400F3017508EF
:10026000E0392E04F500F20A22000C30F0002000E4
:100270000800711C080071102508F400F3017508CE
:10028000E0392F04F500F20A22001030F0002000BF
:100290000800711C080071102608F400F3017508AD
:1002A000E0393004F500F20A22001430F00020009A
:1002B0000800711C080071102708A8080319A22162
:1002C000F400F301F20A0800711C080071102908FB
:1002D000F400F3017116F501F112F20A2200003068
:1002E000F00020000800711C08007112A908031911
:1002F0007116F20108000C190800FA0A7A08013E8A
:10030000031C080022000030F0002000F501FA0173
:100310007112A90803197116F20A08000C1D0800D1
:10032000FA0A7A08F63E031C0800FA01F2010800F6
:100330007608DF39711A20388E0022007008990083
:10034000200008001708F90008002030840023006E
:10035000910115139513151413088000910A840A4E
:1003600033300406031DA929200008007B080B0078
:1003700000340134033407340F341F347B080B007E
:1003800000340A3414341E342834323423009300E9
:1003900015158B1355309600AA30960095148B17BF
:1003A0009518FE33200008006834743474347034B7
:1003B0003A342F342F3470346934633470347234E7
:1003C0006F346A3465346334743473342E346F3468
:1003D000723467342E3475346B34203452346134C3
:1003E0006334653420345334743461347234743477
:1003F000203443346F346E34743472346F346C345C
:100400006C34653472342034563435342034283416
:1004100063342934203450346534743465342034E2
:1004200047347234693466346634693474346834F9
:100430007334203432343034303438342D34323460
:1004400030343134353446342F3457342034523438
:1004500065347634203435342E3432342E3434340A
:1004600020345234653476342034443420345034CB
:10047000433442342034FF3FFF3FFF3FFF3FFF3F05
:10048000FF3FFF3FFF3FFF3FFF3FFF3FFF3FFF3F7C
:10049000FF3FFF3FFF3FFF3FFF3FFF3FFF3FFF3F6C
:1004A000FF3FFF3FFF3FFF3FFF3FFF3FFF3FFF3F5C
:1004B000FF3FFF3FFF3FFF3FFF3FFF3FFF3FFF3F4C
:020000040001F9
:10E00000000000000A000A000A000A000A003200AC
:10E0100000000500150001000100030007000F00CB
:10E020001F0000002000560035002E0032002E0098
:10E03000340020002D002000670072006900640099
:10E040007300740061007200740052006500760075
:10E0500044005F003500320034002E006100730080
:10E060006D002000700069006300700072006F0096
:10E070006A0065006300740073002E006F00720078
:10E0800067002E0075006B002000FF00FF00FF00FE
:10E09000FF00FF00FF00FF00FF00FF00FF00FF0088
:10E0A000FF00FF00FF00FF00FF00FF00FF00FF0078
:10E0B000FF00FF00FF00FF00FF00FF00FF00FF0068
:10E0C000FF00FF00FF00FF00FF00FF00FF00FF0058
:10E0D000FF00FF00FF00FF00FF00FF00FF00FF0048
:10E0E000FF00FF00FF00FF00FF00FF00FF00FF0038
:10E0F000FF00FF00FF00FF00FF00FF00FF00FF0028
:10E10000FF00FF00FF00FF00FF00FF00FF00FF0017
:10E11000FF00FF00FF00FF00FF00FF00FF00FF0007
:10E12000FF00FF00FF00FF00FF00FF00FF00FF00F7
:10E13000FF00FF00FF00FF00FF00FF00FF00FF00E7
:10E14000FF00FF00FF00FF00FF00FF00FF00FF00D7
:10E15000FF00FF00FF00FF00FF00FF00FF00FF00C7
:10E16000FF00FF00FF00FF00FF00FF00FF00FF00B7
:10E17000FF00FF00FF00FF00FF00FF00FF00FF00A7
:10E18000FF00FF00FF00FF00FF00FF00FF00FF0097
:10E19000FF00FF00FF00FF00FF00FF00FF00FF0087
:10E1A000FF00FF00FF00FF00FF00FF00FF00FF0077
:10E1B000FF00FF00FF00FF00FF00FF00FF00FF0067
:10E1C000FF00FF00FF00FF00FF00FF00FF00FF0057
:10E1D000FF00FF00FF00FF00FF00FF00FF00FF0047
:10E1E000FF00FF00FF00FF00FF00FF00FF00FF0037
:10E1F000FF00FF00FF00FF00FF00FF00FF00FF0027
:020000040001F9
:04000E00440FFC1887
:020000040001F9
:08000000FF3FFF3FFF3FFF3F00
:00000001FF
